:020000020000FC
:1000000000C000C00FED0DBF09E109B952E004E0E6
:1000100007BB03E008BBE199FECF01E00EBBE09A0D
:100020005DB2E199FECF02E00EBBE09A6DB2C298DC
:1000300037D25BD00FC0F3E0E0EB92D0D5D0F0E048
:10004000E52F3083D7D006C00894F4D1F3E0E8EF71
:1000500087D000C02AE370D020E26ED020E26CD0BE
:10006000B19903C007D252E04AC0549A5F9BF8CFBF
:100070001CB154981F3241F31F33B9F11032D9F239
:100080001D30E9F11132A1F11F7D143439F11D3415
:1000900031F1143519F01335A1F1DCCF1FD2362D13
:1000A00094D020E249D0F3E0E0EB5AD09DD0532E1B
:1000B00020E242D099D0632E01E0E199FECF0EBB41
:1000C0005DBAF894E29AE19A02E0E199FECF0EBBA4
:1000D0006DBAF894E29AE19A3FD0BCCFE8C1889417
:1000E000A9D1F3E0E8EE3CD0B5CF4AD0F7D1B2CFFA
:1000F000F3E0E0EC35D0A89508E001BDFFCF7AD061
:10010000A9CFF3E0E0EB2CD06FD0F0E0E52F308307
:1001100020E212D088948ED1F4E0EAE021D041E3CD
:1001200017D0312F46D0F0E0E52F3083089482D1EC
:10013000F3E0E8EE15D08ECF539A5D9BFDCF2CB93E
:1001400053980895549A5F9BFDCF1CB1549808951D
:10015000F9DF212FF1DF0895F3E0E0E901D0089500
:10016000C895002021F0202DE7DF3196F9CF0895C2
:10017000F7DFF2DF0895352F28D020E2DDDF089584
:10018000EBDFEADFF2E0E4E0F3DF0895F3E0E4E838
:10019000E7DF0895432F4695469546954695405D81
:1001A0004A3308F0495F3F70305D3A3308F0395FF9
:1001B000089546FD475F4F7036FD375F3F70440F2F
:1001C000440F440F440F342B0895E4DF242FB4DF91
:1001D000232FB2DF089508E020E3331F08F421E362
:1001E000ABDF0A95C9F70895B3DF412FB1DF312F97
:1001F000E0DF0895B1DFF0E0E52F3081E6DF20E2B7
:100200009BDF0895445320496E746572666163658F
:10021000207465737420746F6F6C203033204E6FC0
:1002200076656D6265722032303032204469636BCE
:100230002043617070656C730A0D0A0D5370616321
:100240006520626172203D20456E74657220766182
:100250006C7565200A0D4D206F72206D203D205376
:10026000656E642076616C756520617320646174CD
:1002700061200A0D2F202020203D2053656E642030
:1002800076616C756520617320636F6D6D616E645E
:100290000A0D53202020203D2053656E6420766196
:1002A0006C75652066726F6D206B6579626F617227
:1002B0006420746F207265676973746572200A0D1B
:1002C00044202020203D2044756D702072656769B0
:1002D000737465727320302E2E460A0D3C524554BD
:1002E00055524E3E203D205072696E74206C6173F1
:1002F000742076616C7565206275666665720A0D9C
:1003000054206F722074203D205365742044532084
:10031000706F72742064656C617920706172616DB8
:10032000657465720A0D21203D2072657365742025
:10033000636869700A0D3F203D20446973706C61E9
:1003400079206D656E750A0D416C6C206164647274
:1003500065737320616E642076616C7565732061CE
:1003600072652068657861646563696D616C2061A0
:100370006E642061726520627974652077696465B6
:100380000A0D0000416464726573733A2024000012
:100390000A0D00000A0D43757272656E7420646563
:1003A0006C61792076616C7565203D202024000009
:1003B000456E7465722056616C75653A20240000A4
:1003C0004861726477617265207265736574207626
:1003D0006961207761746368646F6720696E69740E
:1003E00069617465642E00002020446174612053AB
:1003F000656E742E0A0D0000436F6D6D616E642092
:1004000053656E742E200A0D0000456E74657220CF
:10041000726567697374657220746F2073656E64AA
:10042000206461746120746F202824302E2E2446AD
:10043000293A000079E0B19BFECFB09BFCCFC09A77
:10044000B89810F0C098B89AC198B99A29D0B998BC
:10045000C19A26D0B199F8CF18F0C09AB89802C0C6
:10046000C098B89AB19BFECFB898C09A221C7A95D2
:1004700011F7089579E0B199FECF8894B09B06C03A
:100480000894C198B99AB099FECF04C0C198B99A9E
:10049000B09BFECFB998C19A221C7A9561F7089556
:1004A000652D362C3A94F1F76A95D9F7089554DE04
:1004B00053DE00E2402E342D6DDE232F3DDE20E2A0
:1004C0003BDE242C0894B6DFD5DF322D7EDE44DE01
:1004D000439400E3401679F73FDEBCCDF3E0E4E956
:1004E0003FDE352D72DE20E227DE362D6EDE2AE07D
:1004F00023DE2DE021DE2AE01FDE2DE01DDE089543
:00000001FF
